:1000000000308B0000308500003086008316C5303C
:10001000810010308500F0308600831285150514AC
:1000200085140A3098009900960197019001961165
:100030006C208A207520A020EC201E2131202A204F
:1000400031202A202A209F0D9F1E18289F0103106F
:100050001F141828DF30930000000000930B2C2899
:10006000080003308A00100800238A019A00083033
:10007000940005119A0D6620031C051560200515D6
:100080006620940B392805116620971E05156020FF
:100090000515662005116620971E051560200515BB
:1000A000662011089A000830940005119A0D662008
:1000B000031C0515602005156620940B55280800C3
:1000C000213093000000930B622808000430930055
:1000D0000000930B68280800180886000510051416
:1000E0001908860085108514080086018511060808
:1000F0008515A2009D01221A9D15A21A1D15221B0D
:100100009D14A21B1D141D089E0001301E02031920
:100110009E0108009B0104309C0086010314860D9B
:100120000310061A9F289B0A861A9F289B0A061B03
:100130009F289B0A861B9F289B0A9C0B8F280800E0
:100140001B1AE8280A301B020318BA2816190800DF
:100150001618B228161496141B0898000A30990035
:10016000382108009618080016101B08990016156B
:10017000212108009619E92896150B301B02031D52
:10018000C52801309E009706E9280A301B02031D8E
:10019000CC2820309706E9280C301B02031DD328F9
:1001A00002309706E9280D301B02031DDA280430BF
:1001B0009706E9280E301B02031DE1280830970638
:1001C000E9280F301B02031DE92810309706E928A3
:1001D0009611961016110800961DF5280B301B027B
:1001E000031DF528C03091000800A00103101F1C5A
:1001F000FD28171CFD281030A0009F1C032920306B
:1002000097186030A0001F1D092930301719703071
:10021000A0009F1D0F29403097198030A0001F1E9D
:1002200015295030171A9030A0001E08A007023080
:100230008A00200800228A0191000800051A1E2960
:1002400008001808A1000310210DA10EA10C210720
:100250001907900040301002031836291008890051
:1002600083160814831208089700080097010800F5
:100270004030100203180800100889001708880091
:1002800083168B1308128811081555308900AA307F
:1002900089008814081183120800831688184E29D3
:0402A00083120800BD
:100400008207113491343134B13419349934393488
:10041000B934123492343234B2341A349A343A340D
:10042000BA344534C5346534E5344D34CD346D3497
:10043000ED344634C6346634E6344E34CE346E344D
:10044000EE345034D0347034E4345834D834783402
:10045000F8345234D2347234F2345A34DA347A34CE
:10046000FA34043484342434A4344C348C342C349E
:10047000AC34063486342634A6340E348E342E340E
:10048000AE34143494343434B4341C349C346C346A
:10049000BC34163496343634B6341E349E343E346E
:1004A000BE345434D4347434F4345C34DC347C34AA
:1004B000EC345634D6347634F6345E34DE347E345E
:1004C000FE345134D1347134F1345934D93479345F
:1004D000F9345334D3347334B3345B34DB347B3486
:1004E000FB34053485342534A5340D348D342D3456
:1004F000AD34073487342734A7341B348F342F347A
:10050000AF34153495343534B5341D349D343D3411
:10051000BD34173497343734B7341F349F343B34E9
:10052000BF345534D5347534F5345D34DD347D3421
:10053000FD345734D7347734F7345F34DF347F34C5
:02054000BB34CA
:100600008207AA34C03480343034F034B03420341B
:10061000E034A0340C34CC348C343C34FC34BC3462
:100620002C34EC34AC340834C83488343834F834DE
:10063000B8342834E834A8340334C334833433342E
:10064000F334B3342334E334A3340F34CF348F344E
:100650003F34FF34BF342F34EF34AF340B34CB345A
:100660008B343B34FB34BB342B34EB34AB340234AB
:10067000C23482343234F234B2342234E234A2341A
:100680000E34CE348E343E34FE34BE342E34EE344A
:10069000AE340A34CA348A343A34FA34BA342A3496
:1006A000EA34003440346034973470344834683469
:1006B0005834783444346434543474344C346C34A2
:1006C0005C347C3442346234523472344A346A3496
:1006D0005A347A3446346634563476344E346E3472
:0206E0005E3486
:02400E00F93F78
:1042000000000000000000000000000000000000AE
:10421000000000000000000000000000000000009E
:10422000000000000000000000000000000000008E
:10423000000000000000000000000000000000007E
:10424000000000000000000000000000000000006E
:10425000000000000000000000000000000000005E
:10426000000000000000000000000000000000004E
:10427000000000000000000000000000000000003E
:00000001FF
